:04000000983100280B
:1000080070082000A2007108A10080312100901E14
:1000180092282000901E9228230019082900EB003E
:1000280023009D1C28281D1219082900EB00230015
:100038001D16013029002707F0000030283DF10087
:100048007008A7007108A80023001D1D3C289D13F7
:100058009D17013029002707F0000030283DF100E6
:100068007008A7007108A800230019082900EB00F0
:1000780029006B080D3A03194B2827003B08003C60
:10008800031D48283A083E3C031C4B2875280130BC
:100098002900A9000030AA0027003B08003C031DE6
:1000A80057283A083E3C03185E2802302900A90068
:1000B8000030AA0021009012AB3027003A078600D2
:1000C80004303B3D870081013A082100E200270007
:1000D8003B082100E3002700BA01BB012900EB011E
:1000E8009228AB3027003A07860004303B3D870052
:1000F80029006B08810027003A082100E200270048
:100108003B082100E300013027003A07F0000030E7
:100118003B3DF1007008BA007108BB0020002208BE
:08012800F0002108F1000900BC
:100130002A005508033A031D9D285508043A031D5B
:10014000A1285508053A031DA5285508063A031DA0
:04015000A9280800D2
:1001540023009E18AF280000AA282A00550823006F
:040164009A000800F5
:1001680023009E18B9280000B4282A005508230047
:040178009A000800E1
:0A017C0071088A0070088200080074
:1001860024001419D0281F301605F1007108003A12
:0E019600031DD0280130F000D128F001080030
:1001A400200010102A004F08240091002000350878
:1001B4002A00D000200036082A00D1002000370889
:1001C4002A00D200200038082A00D3002400141D7D
:1001D400112920003508360437043804031910297E
:1001E4002A005008510452045304031D092927000E
:1001F4003808860039088700043081004131360808
:10020400F0003708F100BE200130F0005129013020
:100214002A00D0020030D13BD23BD33BE828200057
:1002240035082A00D000200036082A00D10020001A
:1002340037082A00D200200038082A00D300200002
:100244001018492935083604370438040319482995
:100254002A005008510452045304031D4129270065
:100264003808860039088700043081004131360897
:10027400F0003708F100BE200130F00051290130B0
:100284002A00D0020030D13BD23BD33B21292400A9
:10029400161B4E29F001512916150230F0000800F2
:1002A400200035082A00D100200036082A00D20098
:1002B400200037082A00D300200038082A00D40080
:1002C400CF01D0015008123C031D6A294F088E3C0F
:1002D400031C7629C32070080319712976292A0082
:1002E400CF0A0319D00A64292A0012305002031DD0
:1002F4007D298F304F02031C82297B30F000AE2908
:10030400240016142400161CAD29200035083604D8
:10031400370438040319AC292A0051085204530441
:100324005404031DA52927003808860039088700CE
:100334000530810041313608F0003708F100BE2055
:100344000130F000AE2901302A00D1020030D23B46
:0A035400D33BD43B8429F0010800DC
:10035E0024001419BC291F301605F1007108003A4B
:0E036E00031DBC290130F000BD29F00108007C
:06037C0024001615080024
:100382002000F801F9011030FC00710DF80DF90D93
:100392007408F8027508031C750FF9020318D829AE
:1003A2007408F80775080318750FF9070310F00DA4
:0803B200F10DFC0BC629080047
:1003BA00522170082700BC00AF217008003A031DC3
:1003CA00E729E129290026082A00CF00D22070084F
:1003DA002700BD00AF217008003A031DF529EF2957
:1003EA0040302A00CF00D22070082700BD00AF217C
:1003FA007008003A031D022AFC292A004808CF0087
:10040A00D22070082700BF00AF217008003A031DF0
:0E041A000F2A092AFF302700C000BE2108006B
:100428002A00CC0105304C020318242A4C084A073C
:10043800860000304B3D870020308100CC0A162A08
:100448004C084A07860000304B3D87008101CC03E9
:100458004C084A07CD0000304B3DCE000A30F4006E
:10046800F5014808F0004908F100C1217808F000BA
:100478007908F1003030F0072A004D0886004E0850
:100488008700700881000A30F400F5014808F00080
:100498004908F100C12170082A00C8007108C90084
:1004A80000307106031D5A2A00307006031D5D2AAC
:0804B8005F2ACC032C2A080086
:1004C0002000FB01FA01F9018030F800F10CF00C7A
:1004D000031C732A7408F90775080318750FFA07C7
:1004E0000318FB0A0310F01F7B2A7408FA0775082B
:1004F0000318750FFB07FB0CFA0CF90CF80C031C26
:10050000662A7B08F3007A08F2007908F10078087F
:04051000F0000800EF
:10051400553023009600AA30960095140000000080
:020524000800CD
:100526002000FB01FA01F901F801A001730DF80D95
:100536007408F8027508031C750FF9027608031C87
:10054600760FFA027708031C770FFB020001031CE3
:100556000130A002F30D0730FC00730DF80DF90D04
:10056600FA0DFB0DA00D7408731CCB2AF802750852
:10057600031C750FF9027608031C760FFA0277083A
:10058600031C770FFB020001031C0130A002DC2ACA
:10059600F80775080318750FF90776080318760F1C
:1005A600FA0777080318770FFB07000103180130D5
:1005B600A007F30DFC0BB02A720DF80DF90DFA0D1C
:1005C600FB0DA00D7408731CFA2AF8027508031CAB
:1005D600750FF9027608031C760FFA027708031CDA
:1005E600770FFB020001031C0130A0020B2BF8075A
:1005F60075080318750FF90776080318760FFA07BA
:1006060077080318770FFB07000103180130A007CE
:10061600F20D0730FC00720DF80DF90DFA0DFB0D09
:10062600A00D7408721C292BF8027508031C750F9F
:10063600F9027608031C760FFA027708031C770F77
:10064600FB020001031C0130A0023A2BF8077508D3
:100656000318750FF90776080318760FFA07770857
:100666000318770FFB07000103180130A007F20DEE
:10067600FC0B0E2B710DF80DF90DFA0DFB0DA00DEF
:100686007408721C582BF8027508031C750FF902C2
:100696007608031C760FFA027708031C770FFB0215
:1006A6000001031C0130A002692BF8077508031826
:1006B600750FF90776080318760FFA0777080318F7
:1006C600770FFB07000103180130A007F10D073073
:1006D600FC00710DF80DF90DFA0DFB0DA00D740857
:1006E600711C872BF8027508031C750FF902760832
:1006F600031C760FFA027708031C770FFB02000132
:10070600031C0130A002982BF80775080318750F13
:10071600F90776080318760FFA0777080318770F94
:10072600FB07000103180130A007F10DFC0B6C2B31
:10073600700DF80DF90DFA0DFB0DA00D7408711C66
:10074600B62BF8027508031C750FF9027608031C10
:10075600760FFA027708031C770FFB020001031CD1
:100766000130A002C72BF80775080318750FF907A3
:1007760076080318760FFA0777080318770FFB0732
:10078600000103180130A007F00D0730FC00700DC2
:10079600F80DF90DFA0DFB0DA00D7408701CE52B74
:1007A600F8027508031C750FF9027608031C760F0C
:1007B600FA027708031C770FFB020001031C0130C5
:1007C600A002F62BF80775080318750FF9077608C7
:1007D6000318760FFA0777080318770FFB0700014F
:1007E60003180130A007F00DFC0BCA2B7018092C5A
:1007F6007408F80775080318750FF90776080318C3
:0E080600760FFA0777080318770FFB07080034
:10081400522170082700BC00AF217008003A031D64
:10082400142C0E2C290026082A00CF00D220700890
:100834002700BE00AF217008003A031D222C1C2C97
:1008440080302A00CF00D22070082700C000AF21DA
:100854007008003A031D2F2C292C2A004808CF00C9
:10086400D22070082700C100AF217008003A031D90
:0E0874003C2C362CBE21FF302700C2000800AD
:0E0882006730FD00FD0B432C00000000080055
:100890002A004808393C031C542C30304802031C01
:0C08A000542C0130F000552CF001080031
:1008AC000330FC009530FD00FD0B5A2CFC0B5A2C30
:0208BC00080032
:1008BE00FB09FA09F909F809F80A0319F90A0319E3
:0808CE00FA0A0319FB0A0800F5
:0C08D6004230FD00FD0B6D2C00000800FE
:0A08E2000000000000000000080004
:1008EC007408F8027508031C750FF9027608031CCE
:1008FC00760FFA027708031C770FFB02F30D073013
:10090C00FC00730DF80DF90DFA0DFB0D7408731C3A
:10091C009D2CF8027508031C750FF9027608031C50
:10092C00760FFA027708031C770FFB02AA2CF80744
:10093C0075080318750FF90776080318760FFA0770
:10094C0077080318770FFB07F30DFC0B872C720D40
:10095C00F80DF90DFA0DFB0D7408731CC32CF8027D
:10096C007508031C750FF9027608031C760FFA0242
:10097C007708031C770FFB02D02CF80775080318B7
:10098C00750FF90776080318760FFA07770803181E
:10099C00770FFB07F20D0730FC00720DF80DF90D07
:1009AC00FA0DFB0D7408721CE92CF8027508031C77
:1009BC00750FF9027608031C760FFA027708031CF0
:1009CC00770FFB02F62CF80775080318750FF9075B
:1009DC0076080318760FFA0777080318770FFB07CA
:1009EC00F20DFC0BD32C710DF80DF90DFA0DFB0D5E
:1009FC007408721C0F2DF8027508031C750FF90290
:100A0C007608031C760FFA027708031C770FFB029B
:100A1C001C2DF80775080318750FF90776080318CD
:100A2C00760FFA0777080318770FFB07F10D0730DD
:100A3C00FC00710DF80DF90DFA0DFB0D7408711C0D
:100A4C00352DF8027508031C750FF9027608031C86
:100A5C00760FFA027708031C770FFB02422DF8077A
:100A6C0075080318750FF90776080318760FFA073F
:100A7C0077080318770FFB07F10DFC0B1F2D700D7A
:100A8C00F80DF90DFA0DFB0D7408711C5B2DF802B5
:100A9C007508031C750FF9027608031C760FFA0211
:100AAC007708031C770FFB02682DF80775080318ED
:100ABC00750FF90776080318760FFA0777080318ED
:100ACC00770FFB07F00D0730FC00700DF80DF90DDA
:100ADC00FA0DFB0D7408701C812DF8027508031CAF
:100AEC00750FF9027608031C760FFA027708031CBF
:100AFC00770FFB028E2DF80775080318750FF90791
:100B0C0076080318760FFA0777080318770FFB0798
:100B1C00F00DFC0B6B2D7018A12D7408F8077508DF
:100B2C000318750FF90776080318760FFA0777087C
:080B3C000318770FFB07080006
:100B44002A0038088400390885000008F00070087D
:100B54000319B82D38088400390885000008D50029
:100B6400B4202A00B80A0319B90AA22D0630FD00E0
:080B7400FD0BBA2D0000080082
:100B7C002A00BB0138088400390885000008BA0037
:100B8C003A08003A0319D82D3A08D500AA202A00B1
:100B9C00BB0A3B08380784000030393D850000084B
:060BAC00BA00C62D08008E
:0C0BB20024001413941338309500080040
:100BBE002A003808230091002A00390823009200E9
:100BCE0015131514000000001308F0001408F100AE
:020BDE0008000D
:100BE0000B082A00BC008B1323001515151395164E
:100BF0002A003808230091002A00390823009200B7
:100C00002A00BD011F303D020318232E3A0884003C
:100C10003B08850000082300930001310008940080
:100C200002302A00BA070030BB3D8A22013011078A
:100C3000F0000030123DF100700891007108920040
:100C40002A00BD0A022E230095122A003A088400C9
:100C50003B08850000082300930001310008940040
:100C60008A2215112A00BC1B372E8B13382E8B17A6
:020C700008007A
:100C72008230FC00DD30FD00FD0B3D2EFC0B3D2ED5
:060C820000000000080064
:100C88000D302A00D500B4200A302A00D500B4203F
:020C9800080052
:100C9A002A003908F000F036F036F036F0366830BF
:100CAA0084009E308500700884070318850A0008AE
:100CBA00F0003A0886003B0887007008810001307E
:100CCA003A07860000303B3D87000F303905F000B7
:100CDA00683084009E308500700884070318850AEE
:100CEA000008F0007008810002303A0786000030E0
:100CFA003B3D87003808F000F036F036F036F03623
:100D0A00683084009E308500700884070318850ABD
:100D1A000008F0007008810003303A0786000030AE
:100D2A003B3D87000F303805F000683084009E3064
:100D3A008500700884070318850A0008F000700807
:100D4A00810004303A07860000303B3D870081016C
:020D5A0008008F
:100D5C002A00BE01BF013808C0003908C10080302C
:100D6C003906F00080307002031DBE2E00303802B0
:100D7C000318CC2E0130BE000030BF003808003CF8
:100D8C00C0003908031C013EC101C1024008C80063
:100D9C004108C9003A08CA003B08CB0014220630AF
:100DAC00BC000030BD003D08003C031DDF2E3C089C
:100DBC00003C0318FA2E3C083A0786003D083B3DE0
:100DCC00870001303C02F00000303D3BF100700820
:100DDC003A07840071083B3D850000088100013012
:100DEC00BC020030BD3BD92E3A0886003B08870078
:100DFC00203081003E083F040319202FBC01BD01A7
:100E0C003C083A0784003D083B3D85000008203A29
:100E1C00031D142FBC0A0319BD0A062F0130BC0296
:100E2C000030BD3B3C083A0786003D083B3D87003F
:060E3C002D3081000800CA
:0E0E420055303C008F00AA308F000F100800C2
:100E500023009E1690309D002000901E332F23000B
:080E60001908F0002C2F080016
:100E68002A003908B03EC8000A240F302A00380585
:100E7800C8000A24F0302A003805C800C836C83629
:0A0E8800C836C83648160A240800D0
:100E92002A003808F2003908F3007208F0007308DB
:100EA200F100F20A0319F30A700884007108850040
:100EB200000803195D2F4E2F38087202F00039081E
:0E0EC200733BF1000130F0020030F13B0800FC
:100ED0002A0038088400390885000008BA00BB01E0
:100EE0000030BB0000303B06031D782F20303A064F
:100EF0000319832F00303B06031D802F09303A066B
:100F00000319832F872FB80A0319B90A682FBC0168
:100F1000BD01BE01BF0100303B06031D912F2D30E6
:100F20003A06031D9A2FBE0A0319BF0AB80A03190D
:100F3000B90AA52F00303B06031DA02F2B303A061F
:100F4000031DA52FB80A0319B90A38088400390807
:100F500085000008BA00BB010030BB003A08C80099
:100F6000482470080319CE2F3C08F0003D08F1001A
:100F70000A30F4000030F500602230302A003A02D6
:100F8000F20000303B3BF30072087007BC007308AE
:100F9000713DBD00B80A0319B90AA52F3E083F04E8
:100FA0000319DB2F3C08003CF0003D08031C013E08
:100FB000F101F102DF2F3C08F0003D08F1000800CC
:0E0FC00055303C008F00AA308F000F1408003F
:100FCE000330FB000830FC007730FD00FD0BED2FE9
:0A0FDE00FC0BED2FFB0BED2F0800BC
:100FE8000230FC004B30FD00FD0BF82FFC0BF82FF6
:020FF8000800EF
:101000002A0038082300E8002A0039082300E900F4
:101010002A003A082300EA002A003B082300EB00DC
:101020002A003C082300EC002A003D082300ED00C4
:101030002A003E082300EE002A003F082300EF00AC
:101040002A0040082300E0002A0041082300E100B4
:101050002A0042082300E2002A0043082300E3009C
:101060002A0044082300E4002A0045082300E50084
:101070002A0046082300E6002A0047082300E7006C
:02108000080066
:101082002A003A08F1000130F000710803194C28D7
:10109200F035FF3E47287008BC00F009380884008C
:1010A2003908850070088005803084077008800543
:1010B2008031562488313C0880048030840280319B
:1010C200412488313C080005BB003B08003A01304E
:1010D20003190030BB008031562488313B08F000F0
:0210E200080004
:1010E4002A00380884003908850000083A06031DE0
:1010F40080283808F0003908F10092283808F000F8
:101104003908F100B80A0319B90A70088400710893
:1011140085000008F0007008031D7228F001F10139
:021124000800C1
:101126002A00BE01BF0100303F02031D9C280A3081
:101136003E020318AA283E083C0786003F083D3DAC
:10114600870020308100BE0A0319BF0A96283E0890
:101156003C0786003F083D3D870081010130BE0205
:101166000030BF3B3E083C07C0003F083D3DC10084
:101176000A30F400F501F601F7013808F0003908E5
:10118600F1003A08F2003B08F300803193228831DF
:101196007808F0007908F1007A08F2007B08F3007D
:1011A6003030F0072A0040088600410887007008A2
:1011B60081000A30F400F501F601F7013808F00065
:1011C6003908F1003A08F2003B08F3008031932217
:1011D600883170082A00B8007108B9007208BA0090
:1011E6007308BB000030F4007306031D042974085D
:1011F6007206031D042974087106031D042970086C
:10120600003A031D07290C290130BE020030BF3BFE
:04121600B5280800EF
:10121A002A003A08F1000130F00071080319182970
:10122A00F035FF3E13297008BE007009BD00BC01ED
:10123A003808840039088500BB013B08073C031CB9
:10124A004F293D088005803084073D08800580319C
:10125A00712488313E0880048031712488318030BD
:10126A0084023E080005F000031947293B08F100F3
:10127A000130F000710803194529F035FF3E402975
:10128A007008BC0480316B24883180316B2488312A
:0A129A00BB0A22293C08F0000800FE
:1012A4002A003808F4003908F50074088400750829
:1012B4008500000803196229F40A0319F50A57295D
:1012C4007408F2007508F300F40A0319F50A3A08E1
:1012D400F0003B08F100BA0A0319BB0A7008840045
:1012E4007108850072088600730887000008810071
:1012F4007208840073088500000803198229622992
:0A1304003808F0003908F100080075
:10130E0020002230FC00F801F901FA01FB01FC0378
:10131E000319BC290310FB0CFA0CF90CF80CF30C96
:10132E00F20CF10CF00C031C8E29FC030319AE29F0
:10133E007408F80775080318750FF907760803186F
:10134E00760FFA0777080318770FFB0792297408B0
:10135E00F80775080318750FF90776080318760F46
:0C136E00FA0777080318770FFB07080048
:10137A002A003A08F1000130F00071080319C8295F
:10138A00F035FF3EC3297008BE00F0097008BD00A1
:10139A003808840039088500700880058030840781
:1013AA00BC013C08073C031CF1293C08F0003B083F
:1013BA00F10070080319E429F136FF3EDF293D08E0
:1013CA008005711CEA293E08800480314124883155
:1013DA003E088004BC0AD6298030840280316B24FE
:0A13EA00883180316B24883108003F
:1013F40020302A00C80080310A2488312A00C8011C
:1014040080310A24883121302A00C80080310A241E
:1014140088312A003808C80080310A2488312A001B
:1014240038080F3EC80080310A24883122302A004F
:10143400C80080310A24883101302A00C800803174
:101444000A24883103302A00C80080310A248831F4
:101454002A00BA01BB0180303B06F00080307002E4
:10146400031D362A30303A020318582A3908F0008E
:10147400F101F035F10D4130700784000030713D09
:1014840085000008F00001310008F1003A087007F7
:1014940084003B08713D85000008C8008031DD21CF
:0E14A40088312A00BA0A0319BB0A2D2A080053
:1014B2002A003C08F000BC03700803198E2A380881
:1014C2008400390885000008003A0319772A3A088F
:1014D20084003B0885000008F100380884003908C0
:1014E200850000087106031D772A872A38088400C0
:1014F200390885000008F0003A0884003B0885009E
:101502000008F002F1010030F13B902AB80A0319F9
:10151200B90ABA0A0319BB0A592AF001F1010800F3
:101522000B082A00BA008B133808230091002A0006
:1015320039082300920015131516151580318A22D9
:10154200883115112A00BA1BA82A8B13A92A8B17D6
:0215520008008F
:101554007408003A031DC32A7508003A031DC32A00
:101564007608003A031DC32A7708003A031DC32AEC
:10157400FF30F000FF30F100FF30F2007F30F30065
:101584005F2B2000FC01F71BFC0AFD01FB01FA01A3
:10159400F901F80173087204710470040319582BDB
:1015A40073087706A000A01BFD09F71FE42AF409BD
:1015B400F509F609F709F40A0319F50A0319F60AF5
:1015C4000319F70AF31FF12AF009F109F209F309E3
:1015D400F00A0319F10A0319F20A0319F30A73084A
:1015E4007704A000A01B142B803176248831FC1BC7
:1015F400312BFD1F582BF009F109F209F309F00A08
:101604000319F10A0319F20A0319F30AF809F9098B
:10161400FA09FB09F80A0319F90A0319FA0A031962
:10162400FB0A582BF71F2B2BF31B252B7308FB00EE
:101634007208FA007108F9007008F800F301F20169
:10164400F101F001FB2AF301F201F101F001F00ACA
:101654000034F309F209F109F009FC17F62AF80A33
:101664000319F90A0319FA0A0319FB0A7408780220
:10167400031DFB2A75087902031DFB2A76087A02EA
:10168400031DFB2A77087B02031DFB2AFB01FA01D9
:10169400F901F801F00A0319F10A0319F20A03190E
:1016A400F30AF31FFB2AA0012016FF34A0017C1CBF
:0C16B4005E2B80315F248831003E08006E
:1016C00029006C08F000F036F036F036F03668305D
:1016D00084009E308500700884070318850A00087E
:1016E000F0006D0886006E088700700881000130E8
:1016F0006D07860000306E3D87000F306C05F000EE
:10170000683084009E308500700884070318850ABD
:101710000008F0007008810002306D07860000307C
:081720006E3D87008101080005
:101728002900A701A801230019082900EB00EB01F3
:1017380023001D162900A901AA0121009016AB302B
:1017480027003A07860004303B3D870081013A08AC
:101758002100E20027003B082100E3002700BA012E
:08176800BB012900EB010800A0
:1017700021302A00C80080310A2488312A00C8019B
:1017800080310A2488317F302A00C80080310A2441
:10179000883122302A00C80080310A2488312A008A
:1017A000C80180310A24883103302A00C800803102
:1017B0000A248831D3302A00C80080310A248831B5
:1017C00040302A00C80080310A2488312A00B8013C
:1017D000B9018031342788312900EC0104306C02D2
:1017E00003181E2C6C08B03E2A00C80080310A2461
:1017F000883101302A00C80080310A248831103035
:101800002A00C80080310A2488310D30FD00FD0B0C
:10181000072C2900ED0180306D0203181C2C2A00D2
:10182000C8018031DD2188311A30FD00FD0B162CF6
:1018300000002900ED0A0B2CEC0AEE2B2E302A00BA
:10184000C80080310A2488312A00B801B9018031EA
:0618500034278831080076
:1018560056302A00B8009E30B9008031A225883162
:101866008030B8001F30B9008031DF25883170081C
:101876002900EC007108ED0070082A00B800710814
:10188600B9002030BA000130BB0080314D268831C6
:101896002030B8000130B9008031BE258831803152
:1018A60044268831803029006D06F00080303F3AAA
:1018B6007002031D602CFF306C020318822D163057
:1018C6002A00B8009E30B9008031A2258831200058
:1018D600EE01EF01A0302100E0000130E100290017
:1018E600EE01EF0180306F06F00080307002031DBC
:1018F6007E2C05306E020318DB2C80306E072A0022
:10190600B8001F3029006F3D2A00B9008031DF255D
:10191600883170082900EC007108ED00A030200025
:101926006E07860001306F3D8700FF30F0057008B6
:101936008100A0306E07840001306F3D85000008ED
:101946002A00D5008031AA208831013020006E0798
:10195600F00000306F3DF100A030700786000130C6
:10196600713D870029006D08F0000030ED1BFF3047
:10197600F10070088100013020006E07F000003091
:101986006F3DF100A030700784000130713D850085
:1019960000082A00D5008031AA20883102302000B4
:1019A600EE070030EF3D2900EE0A0319EF0A752C09
:1019B6002300A501A0302A00B8000130B90080310B
:1019C6004927883170082100E6007108E700A03039
:1019D600E0000130E100600884006108850000082D
:1019E6002D3A0319072D6008840061088500000858
:1019F6002D3A0319072D6008840061088500000848
:101A0600203A0319072D792D2900EC01ED01EE018D
:101A1600EF0180306F06F00080307002031D152D37
:101A260007306E020318322D6E082100600784000D
:101A360029006F082100613D850000082A00C800C2
:101A4600803148248831700803192D2D2900EC0AAD
:101A56000319ED0A2900EE0A0319EF0A0C2D2100DD
:101A660066082900EC00210067082900ED00210026
:101A7600660867040319702D60082A00B800210063
:101A860061082A00B9008031682788317008210072
:101A9600E8007108E900E5302A00B8009E30B90078
:101AA6008031A2258831210068082A00B80021006B
:101AB60069082A00B9002030BA000130BB00803125
:101AC600AE2688312030B8000130B9008031BE25FD
:101AD6008831803144268831782DEE302A00B800CE
:101AE6009E30B9008031A2258831812D2A003130FF
:101AF600B8009E30B9008031A22588318A2D2A008F
:101B0600B330B8009E30B9008031A2258831080074
:101B16000E302A00B8000030B900BA0141200E305C
:101B2600B8000030B900BA01CC30BB00BD210E3080
:101B3600B8000030B900BA014430BB00BD21803185
:101B4600E72788310E30B8000030B900BA014120CD
:101B56000E30B8000030B900BA01CC30BB00BD2150
:101B66000E30B8000030B900BA01BE30BB00BD214E
:101B76008031E72788310E30B8000030B900BA014D
:101B86000D2170082000BF00C0010E302A00B800E9
:101B96000030B900BA010D2170082000BA00B90161
:0A1BA6003F08B9074008BA3D0800E7
:101BB0000B30FB002630FC005D30FD00FD0BDE2D00
:0E1BC000FC0BDE2DFB0BDE2D000000000800EC
:101BCE002900EE01EF012A002008A6002108A70037
:101BDE002208A8002308A90080302306F0008030D8
:101BEE007002031D042E00302202031D042E00304D
:101BFE002102031D042E003020020318182E01307E
:101C0E002900EE000030EF002A00A601A701A8016E
:101C1E00A9012008A6022108A73B2208A83B2308F9
:101C2E00A93B2608B8002708B9002808BA002908D9
:101C3E00BB002408BC002508BD0093200B302900F2
:101C4E00EC000030ED006D08003C031D302E6C08DA
:101C5E00003C0318512E6C082A0024078600290028
:101C6E006D082A00253D8700013029006C02F00026
:101C7E0000306D3BF10070082A00240784007108C3
:101C8E00253D85000008810001302900EC0200305E
:101C9E00ED3B2A2E2A0024088600250887002030D6
:101CAE00810029006E086F040319812EEC01ED01ED
:101CBE006C082A002407840029006D082A00253D9F
:101CCE0085000008203A031D712E2900EC0A031925
:101CDE00ED0A5F2E29000130EC020030ED3B6C085E
:101CEE002A002407860029006D082A00253D87005A
:061CFE002D3081000800FA
:101D04002900EE01EF016C08F3006D08F4006C0883
:101D1400F5006D08F6007308840074088500000857
:101D2400203A031D9A2E6E086F04031D9A2EAB2EC3
:101D34000130EE000030EF00730884007408850061
:101D4400750886007608870000088100F50A0319E3
:101D5400F60A7308F1007408F200F30A0319F40A8E
:101D640071088400720885000008003A031D8D2E56
:0A1D74006C08F0006D08F100080093
:101D7E002A00A501A6012008B8002108B90080316B
:101D8E0034278831562F642F642F2A002208B8007A
:101D9E002308B90080314927883170082900EE00E8
:101DAE007108EF008030F200803071067202031D60
:101DBE00E22E7008003C0318542F2A00A601803032
:101DCE00F000803029006F067002031DF12E6E08A0
:101DDE002A0026020318542F2A000730260729004E
:101DEE00EC00ED010030ED3D6E08EC026F08ED3BAE
:101DFE000430F00070080319082FEC35ED0DFF3E8E
:101E0E00022F2A002608220784000030233D850079
:101E1E000008F1007108A50071082F3C0318242F4B
:101E2E003A3025020318242F29006C082A00B80026
:101E3E0030302502B900FA21522F452F29006C08A7
:101E4E002A00B8000A30B900FA21522F29006C0876
:101E5E002A00B8000B30B900FA21522F29006C0865
:101E6E002A00B8000C30B900FA21522F29006C0854
:101E7E002A00B8000B30B900FA21522F25082E3A4D
:101E8E000319252F2508203A03192D2F2508B03ABE
:101E9E000319352F3D2FA60AE62E642F642F2A0034
:101EAE002408013A0319CA2E2408023A0319CB2E2C
:0C1EBE002408033A0319CC2E552F08000D
:101ECA00003029006D06031D6C2F00306C060319C3
:101EDA00B92F6C0884006D08850000080319B92F12
:101EEA006E082A00B80029006F082A00B90080315C
:101EFA00492788317008BC0029006C082A00B800FC
:101F0A0029006D082A00B90029006E082A00BA00C3
:101F1A0029006F082A00BB00592200307106031DF0
:101F2A00982F00307006031DA02F29006C08F000BE
:101F3A006D08F100BB2F290001306C072A00B80098
:101F4A00003029006D3D2A00B90029006E0884007E
:101F5A006F08850000082A00BA007220700829005C
:0E1F6A00EC007108ED00652FF001F101080098
:101F78001530FB004B30FC00BE30FD00FD0BC22FBE
:0C1F8800FC0BC22FFB0BC22F0000080056
:101F940029006E0884006F0885000008F0007008AE
:101FA4000319E72F6E0884006F0885000008F0000D
:101FB4006C0886006D08870070088100EC0A03191C
:101FC400ED0AEE0A0319EF0ACA2F6C0886006D08A1
:061FD400870081010800F6
:101FDA00210099011917991619169915991498013A
:021FEA000800ED
:101FEC0012001E00F003031DF62FF103031DF62F44
:021FFC000800DB
:10200000210068082A00B800210069082A00B900E8
:102010004430BA002130BB008031AE2690314430CC
:10202000B8002130B9008031492790317008210073
:10203000E6007108E70001307005F2007108F30056
:102040000030F3057308003C031D28287208003C8B
:1020500003183A2844302A00B8002130B900333040
:10206000BA000030BB008831522190312100E60ACD
:102070000319E70AE736E60C44302A00B80021309D
:10208000B9008031BE259031803144269031210045
:1020900066082A00C800210067082A00C90020300D
:1020A000CA000130CB008031142290312030D5009D
:1020B0008031AA20903120302A00B8000130B900C8
:1020C0008031BE25903180314426903178302A000D
:1020D000B8009E30B9008031A22590312900EC0172
:1020E000ED0180306D06F00080307002031D7A280B
:1020F00020306C020318902880306C072A00B8004A
:102100001F3029006D3D2A00B9008831912290319D
:102110008031392690312900EC0A0319ED0A712823
:1021200096302A00B8009E30B9008031A225903147
:102130002900EC01ED012100670829006D02031D53
:10214000A5282100660829006C020318CB288030DE
:102150006C072A00B8001F3029006D3D2A00B90025
:102160004430BA002130BB0029006C08F0006D0833
:10217000F100F035F10D70082A00BA077108BB3D77
:102180008031F02590318031392690312900EC0AD8
:102190000319ED0A9B2880306C072A00B8001F3015
:1021A00029006D3D2A00B900BA01BB018031F0253C
:0421B0009031080062
:1021B4002A0020082000B5002A0021082000B600CB
:1021C4002A0022082000B7002A0023082000B800B3
:1021D4002A0024082700B6002A0025082700B70093
:1021E4002A0026082700B8002A0027082700B9007B
:0221F4000800E1
:1021F6002200961323008C01FF3021008C000C1264
:1022060022000C1623008D01FF3021008D002400D2
:102216008D0125000D160D178D128D13F030260039
:102226008D0027008D0123008E01DF3021008E00F6
:10223600223024008E0021008E148E1225008E1668
:0E22460021008E1222008E1621009513080032
:102254002A0034082400A0002A0035082400A10024
:102264002A0036082400A2002A0037082400A3000C
:102274002A0020082200E4002A0021082200E500A8
:102284002A0022082200E6002A0023082200E70090
:102294002A0024082200E8002A0025082200E90078
:1022A4002A0026082200EA002A0027082200EB0060
:1022B4002A0028082100EA002A0029082100EB004E
:1022C4002A002A082100EC002A002B082100ED0036
:1022D4002A002C082200E0002A002D082200E10038
:1022E4002A002E082200E2002A002F082200E30020
:1022F4002A0030082200EC002A0031082200ED00F8
:102304002A0032082200EE002A0033082200EF00DF
:022314000800BF
:102316008D302A00C80080310A24903114302A00FA
:10232600C80080310A249031AF302A00C8008031BD
:062336000A2490310800AA
:10233C00AE302A00C80080310A2490316830FC008D
:10234C00E430FD00FD0BA829FC0BA8290000AF30E0
:10235C002A00C80080310A2490316830FC00E43037
:10236C00FD00FD0BB729FC0BB7290000B0302A008B
:10237C00C80080310A2490312A00C80180310A2417
:10238C00903103302A00C80080310A24903120306B
:10239C002A00C80080310A24903102302A00C8007B
:1023AC0080310A24903121302A00C80080310A245F
:1023BC0090312A00C80180310A2490317F302A00E4
:1023CC00C80080310A24903122302A00C8008031A4
:1023DC000A2490312A00C80180310A24903103303C
:1023EC002A00C80080310A249031A1302A00C8008C
:1023FC0080310A249031A4302A00C80080310A248C
:10240C009031A6302A00C80080310A249031C8309F
:10241C002A00C80080310A249031D3302A00C80029
:10242C0080310A24903140302A00C80080310A24BF
:10243C009031D5302A00C80080310A249031803088
:10244C002A00C80080310A249031A8302A00C80024
:10245C0080310A2490313F302A00C80080310A2490
:10246C009031D6302A00C80080310A249031803057
:10247C002A00C80080310A249031D9302A00C800C3
:10248C0080310A2490311F302A00C80080310A2480
:10249C009031DA302A00C80080310A249031203083
:1024AC002A00C80080310A249031EE302A00C8007E
:1024BC0080310A24903181302A00C80080310A24EE
:1024CC0090317F302A00C80080310A2490312E30A0
:1024DC002A00C80080310A249031DB302A00C80061
:1024EC0080310A24903140302A00C80080310A24FF
:1024FC0090318D302A00C80080310A24903114307C
:10250C002A00C80080310A249031AF302A00C8005C
:08251C0080310A24903108000F
:102524002A00B801B9018031342790312900EC0127
:10253400ED0100306D02031DA12A04306C02031862
:10254400DC2A8530FD00FD0BA52AEE01EF010030E9
:102554006F02031DAF2A80306E020318D82A073099
:10256400F2006C08F0006D08F10072080319BE2A2D
:10257400F035F10DFF3EB82A6E08F0076F08F13D03
:102584005630700784002230713D850000082A000F
:10259400C8008031DD2190311A30FD00FD0BD02AB6
:1025A40000002900EE0A0319EF0AA92AEC0A03190C
:1025B400ED0A9B2A2A00B801B901803134279031F1
:0225C40008000D
:1025C6002A00A6012900ED1FF82A01302A00A600DC
:1025D60029006E0886006F0887002D308100EC09FF
:1025E600ED09EC0A0319ED0A012B2A00A6012900C0
:1025F6006E0886006F088700203081006C08F000A6
:102606006D08F100F136F00CF136F00CF136F00CF5
:10261600F136F00C70082A00A0007108A100013004
:1026260029006E072A00A700003029006F3D2A0006
:10263600A8000A30F4000030F5008031C121903145
:102646000A30F4000030F5008031C121903178085D
:10265600F0007908F1003030F0072A0027088600DC
:102666002808870070088100013029006E07840061
:1026760000306F3D85000008303A031D4A2B0130BB
:102686006E07860000306F3D8700203081000230E3
:102696006E072A00A700003029006F3D2A00A80017
:1026A6000A30F4000030F5002008F0002108F1009F
:1026B6008031C12190317808F0007908F10030307E
:1026C600F0072A002708860028088700700881007E
:1026D60029006C082A00A20029006D082A00A30020
:1026E600A401A5010F30A2050030A305A405A50588
:1026F600083029006E07860000306F3D8700810193
:102706002A002208F0002308F1002408F200250818
:10271600F3007130F4000230F500F601F70188315C
:102726008721903170082A00A2007108A300720860
:10273600A4007308A500033029006E078600003048
:102746006F3D87002E30810004306E072A00A700F7
:10275600003029006F3D2A00A800E830F40003305D
:10276600F500F601F7012208F0002308F10024081D
:10277600F2002508F3008831AA2290313030F007A4
:102786002A0027088600280887007008810005307F
:1027960029006E072A00A700003029006F3D2A0095
:1027A600A8006430F400F501F601F7012208F000F4
:1027B6002308F1002408F2002508F3008831AA2234
:1027C60090310A30F400F501F601F7018831AA22AA
:1027D60090317808F0007908F1007A08F2007B0859
:1027E600F3003030F0072A00270886002808870003
:1027F60070088100063029006E072A00A700003005
:1028060029006F3D2A00A8000A30F400F501F60100
:10281600F7012208F0002308F1002408F200250839
:10282600F3008831AA2290310A30F400F501F6014E
:10283600F7018831AA2290317808F0007908F10072
:102846007A08F2007B08F3003030F0072A002708E8
:1028560086002808870070088100073029006E0767
:10286600860000306F3D8700810108306E078600C4
:1028760000306F3D870081012A002008F000210802
:10288600F100F201F301E830F4000330F500003006
:10289600F6000030F70088318721903170082A0051
:1028A600A7007108A8007208A9007308AA000A30D8
:1028B600F400F501F601F7012208F0002308F10003
:1028C6002408F2002508F3008831AA229031700806
:1028D6002A0027072000BB0071082A00283D200097
:1028E600BC0072082A00293D2000BD0073082A009A
:1028F6002A3D2000BE002A002608013A031D982C16
:10290600F001F101F201F30120003B08F0023C085E
:10291600F13B3D08F23B3E08F33B7008BB007108F3
:10292600BC007208BD007308BE002A002608F0002D
:02293600080097
:102938008031212790313D00A50194010D309D0083
:1029480012309F0010309E0011309C000E303C0069
:10295800A0000C30A1003D00A50194018031E027C2
:0429680090310800A2
:10296C00AF302400A0000130A1000030A2000030E4
:10297C00A30052302200E4000130E5000030E600F4
:10298C000030E700FF30E800FF30E9000030EA00DB
:10299C000030EB00FF302100EA00FF30EB00FF308D
:1029AC00EC00FF30ED00D2302200E0000030E100FE
:1029BC004F30E2000530E300BE30EC000130ED009A
:1029CC000030EE000030EF0029006C082A00B8003F
:1029DC0029006D082A00B90029006E082A00BA00E7
:1029EC0029006F082A00BB008031D92590310800DE
:1029FC00FF302A00B800FF30B9000030BA000030B8
:102A0C00BB00B430BC000030BD005530BE000530FA
:102A1C00BF00FF30C000FF30C1000030C2000030EA
:102A2C00C300FF30C400FF30C5000030C6000030CA
:102A3C00C700883100209031803128279031080060
:103000001A278831ED2798319031FB209831903183
:103010009C2498312100E401E50180306506F00030
:1030200080307002031D1628063064020318282819
:1030300022008E120C128031E72798318E160C1662
:103040008031E72798312100E40A0319E50A0D28A9
:10305000A0302000DB000030DC0023009F15CF30C3
:103060009B009C011E159031FE249831F9302A00F6
:10307000B8009D30B9008031A22598318031E72712
:10308000983180314426983144302A00B8009E306F
:10309000B9008031A22598312100E401E50180309A
:1030A0006506F00080307002031D58280530640268
:1030B000031874286408F0006508F100F035F10D7C
:1030C0002330700784000030713D850000082A001D
:1030D000B80001310008B9008031A22598312100E3
:1030E000E40A0319E50A4F2822008E16803144268F
:1030F00098318B132100E401E50180306506F00072
:103100008030003A7002031D87283F3064020318A4
:103110009428A030640786000030653D8700810157
:10312000E40A0319E50A7D28A0302000DB00003006
:10313000DC00DC302A00B8009D30B9008031A225C7
:1031400098310A30240092009031B62498310A3028
:103150002A00A000A101A201A3019830A400003020
:10316000A5005530A6000530A7009031DA2098312F
:1031700052302A00A0000130A1000030A20000302F
:10318000A300FF30A400FF30A5000030A6000030EF
:10319000A700FF30A800FF30A900FF30AA00FF30D1
:1031A000AB00D230AC000030AD004F30AE00053087
:1031B000AF00BE30B0000130B1000030B2000030CE
:1031C000B300AF30B4000130B5000030B6000030BD
:1031D000B70090312A21983178302000AF00783044
:1031E0002900A60090319E2198318031E72798313F
:1031F00090318B219831903192229831C0302A0041
:10320000B8009E30B9008031A22598318831B823AA
:1032100098312100E801E90188312B24983180316F
:10322000442698312000EE01EF010E302A00B8004C
:103230000030B900BA018831412098318031F4273B
:1032400098310E30B8000030B900BA013330BB00FD
:103250008831BD2198318031F42798310E30B80083
:103260000030B900BA0188310D2198317008290069
:10327000EB008031F427983187302A00B8009E3067
:10328000B9008031A22598312200A00129006B08E5
:10329000EC002030ED000130EE00883160239831E1
:1032A00020302A00B8000130B9008031BE259831A5
:1032B000F730B8009E30B9008031A2259831210046
:1032C000E401E50180306506F00080307002031DE6
:1032D0006B290630640203189F290E302A00B800BB
:1032E0000030B900BA0188310D21983170082900E9
:1032F000EB008031392698315D302100640786006B
:103300000030653D870029006B0881002200A00184
:1033100029006B08EC002030ED000130EE00883110
:103320006023983120302A00B8000130B900803184
:10333000BE2598312100E40A0319E50A622980318B
:103340004426983122000C168E1620008E18B129C2
:10335000CD302A00B8009E30B9008031A2259831C6
:10336000B9292A00D930B8009E30B9008031A22591
:1033700098318031442698310B178B17883194236C
:1033800098312200A00120008E18CE290E302A008C
:10339000B8009F30B9008031A225983188318B2543
:1033A000983139082900EC0020003A082900ED0086
:1033B0002030EE000130EF009031E32298312030D0
:1033C000B8000130B90080314927983170082000D9
:1033D000EC007108ED00203070072900EC0001308E
:1033E000713DED00FC30EE009730EF008831CA27C8
:1033F000983120008E18042A20302A00B8000130AD
:10340000B9008031BE25983120008E18242A210071
:1034100068082A00B800210069082A00B900203095
:10342000BA000130BB008031AE2698310430B800BC
:103430009F30B9008031A22598312030B80001308A
:10344000B9008031BE25983120008E182D2A163003
:103450002A00D5008031AA2098310A302A00B8000D
:103460009F30B9008031A22598312200A0012100AF
:10347000680820003B072A00A000210069082000FE
:103480003C3D2A00A10000302100E91BFF30200054
:103490003D3D2A00A20000302100E91BFF30200042
:1034A0003E3D2A00A3002030A4000130A500883151
:1034B000E725983120302900EC000130ED008831FB
:1034C00082269831220020082A00D5008031AA20C7
:1034D0009831220021082A00D5008031AA20983195
:1034E0002E302A00D5008031AA20983122302A00BF
:1034F000B8000130B9008031BE259831FD30B800E8
:103500008730B9008031A22598318831B8239831AD
:1035100022002308A4002208A3002E30A2002A00C3
:10352000A001A1012030A2000130A3000330A400BB
:103530008831BF269831FE302A00B8009E30B9008D
:103540008031A22598312100680820003B07F00057
:103550002100690820003C3DF10000302100E91BFA
:10356000FF3020003D3DF20000302100E91BFF301C
:1035700020003E3DF3007C30F0029230F13B003001
:10358000F23BF33B7008E6007108E7007208E800C0
:103590007308E90070082A00A0007108A1007208F1
:1035A000A2007308A3002030A4000130A5008831D8
:1035B000E725983120302900EC000130ED008831FA
:1035C0008226983120302A00B8000130B9008031BD
:1035D000BE25983180314426983188319423983122
:1035E0008831BC2798317F30F00080302000690698
:1035F0007002031D052B6808FF3C031D052B67089F
:10360000FE3C031D052B6608703C0318232B8030FD
:103610006906F00080307002031D182B003068022C
:10362000031D182B01306702031D182B9030660212
:103630000318232B22008E120C128831D8259831C2
:103640008E160C16592B8030F00080302000690651
:103650007002031D352B6808003C031D352B6708DD
:10366000003C031D352B6608FA3C03183E2B220054
:103670008E160C128831D82598310C168030200017
:103680006906F0007F307002031D502BFF30680286
:10369000031D502BFF306702031D502B06306602BE
:1036A0000318592B22000C168E128831D825983118
:1036B0008E16003029002A06031D602B01302906D2
:1036C000031D5F2CAB30EC000430ED003030EE0019
:1036D0000030EF0088316527983170082000EA003B
:1036E0007108EB00023070072A00B8000030713D0D
:1036F000B90080314927983170082000EC0071082A
:10370000ED002100EE01EF0120006B08003C031DDD
:103710008B2B6A08003C03185C2C8030F000803052
:103720006D067002031D962B6C08013C03185C2C7F
:1037300002306A07840000306B3D850000082D3A96
:103740000319B72B02306A07840000306B3D8500F7
:103750000008203A0319B72B02306A0784000030B2
:103760006B3D850000082B3A0319B72B5C2C013008
:103770002100E4000030E50080306506F000803074
:1037800020006D067002031DC82B6C082100640226
:103790000318E72B023020006A07F00000306B3D71
:1037A000F10021006408700784006508713D850000
:1037B00000082A00C8008031482498317008210090
:1037C000EE070030EF3DE40A0319E50ABC2B013097
:1037D00020006C02F10000306D3BF20021006F0808
:1037E0007206031DF52B71086E06031D5C2CA530B7
:1037F0002A00B8009E30B9008031A22598310230ED
:1038000020006A072A00B800003020006B3D2A0023
:10381000B90080316827983170082700B40071081A
:10382000B50070082A00B8007108B9002030BA004D
:103830000130BB008031AE2698312030B800013015
:10384000B9008031BE2598318031442698318030CE
:10385000F43AF0008030270035067002031D322C48
:103860003408483C0318542C80303506F000803072
:103870000B3A7002031D3E2CB83034020318542C4E
:1038800012302A00B8009F30B9008031A22598314B
:10389000270034082100E800270035082100E9004E
:1038A0009031002098315C2C2A00B330B8009D3054
:1038B000B9008031A22598312000EA01EB01C1292D
:0238C000602C7A
:103E340056308400963085003830F0000130F100AF
:103E440023308600003087008831F6279831080037
:060FFA00B0344334003462
:102A4C00203453346F347534723463346534203429
:102A5C003A34203454346834653472346D346F3401
:102A6C006D3465347434723465345F3443346F348C
:102A7C00723470346F34723465346C345F34313486
:102A8C003634463431343634313439345F34553499
:102A9C0041345234543431345F3452344234373448
:102AAC005F34543458345F345234423435345F34E8
:102ABC00523458345F344934323443345F345234F2
:102ACC00423436345F34533443344C345F345234F0
:102ADC00423434345F345334443441345F344434FA
:102AEC005334313438344234323430345F34523429
:102AFC00433432345F3432343034323430345F3433
:102B0C00303434345F34303432342E346334203443
:062B1C000D340A34003400
:102B220020344434693472346534633474346F3419
:102B32007234793420343A34203443343A345C34B5
:102B42005F344D3469346B3472346F3443345C34E3
:102B52005F344D3465347334503472346F346A34B4
:102B62006534743473345F344D3469346B34723485
:102B72006F3443345C345F345434683465347234B3
:102B82006D346F346D3465347434723465345F344B
:102B920043346F34723470346F34723465346C344D
:102BA2005F34323430343234303420340D340A3429
:022BB2000034ED
:102BB4002034503472346F346A34653474342034BD
:102BC4003A34203454346834653472346D346F3498
:102BD4006D3465347434723465345F3443346F3423
:102BE400723470346F34723465346C345F3431341D
:102BF4003634463431343634313439345F344F3436
:102C04004C34453444345F344434533431343834EC
:102C14004234323430345F34323430343034343447
:102C2400303433342E346D34633470347034693456
:062C34000D340A340034E7
:102C3A0020345434653472346D3469346E346134FA
:102C4A006C34203470346F34753472342034643404
:102C5A00693461346C346F346734753465342034C4
:102C6A0065347434203456346934733475342034FA
:102C7A0020346434653472346F3475346C3465349A
:102C8A006D3465346E3474342034703472346F3475
:102C9A006734723461346D346D3465340D340A34FA
:022CAA000034F4
:102CAC00DE34973491349534DA34953426349534B3
:082CBC0084349D341D3496346C
:022CC400783462
:062CC6004B343D340034E4
:042CCC00203400347C
:082CD00000340034003400342C
:042CD8000034003490
:082CDC00003400340034003420
:042CE4000034003484
:102CE80064349C3494349C34AE3497344E349734E2
:102CF8007E34973454349D3424349D34C4349C3405
:102D0800F4349C34BE3496348E3496341E3497345E
:042D1800EE349634CB
:102D1C000034003400340034003400340034003407
:102D2C0000340034003400340034003400340034F7
:102D3C0000340034003400340034003400340034E7
:102D4C0000340034003400340034003400340034D7
:102D5C0000340034003400340034003400340034C7
:102D6C0000340034FF34FF34FF34FF3400340034BB
:102D7C000034E034F834FC34FE34FF341F340F34A8
:102D8C000F340F341F34FE34FE34FC34F0348034F2
:102D9C00003407340F343F343F347F347C34783480
:102DAC00783478343C34FF34FF34FF34FF34FF3450
:102DBC0000340E343E347E347E34FE34F834F03439
:102DCC00F034F0347C347F343F341F340F3401340E
:102DDC0000340034003400341F34E0340034003448
:102DEC00003400341834C03400340034003400345F
:102DFC001834C03400340034003400341F34C03470
:102E0C000034003400340034003400340034003416
:102E1C000034003400340034003400340034003406
:102E2C0000340034003400340034003400340034F6
:102E3C0000340034003400340034003400340034E6
:102E4C0000340034003400340034003400340034D6
:102E5C0000340034003400340034003400340034C6
:102E6C0000340034003400340034003400340034B6
:102E7C0000340034003400340034003400340034A6
:102E8C000034003400340034003400340034003496
:102E9C000034303478347E347E347F341F340F3435
:102EAC000F341F34FF34FE34FE34FC34F034003461
:102EBC0000340034003400340034003400340E3458
:102ECC000E340F341F34FB34FB34F934F034C0347B
:102EDC00003406341F343F347F347F34FC34F034F8
:102EEC00F034F034FC347F347F343F341F340734F7
:102EFC0000340034003400340034C034E034F8348E
:102F0C00FC34FF34FF34FF34FF34FF34003400341E
:102F1C00C034E034F834FC34FF34BF348F348334A1
:102F2C008134FF34FF34FF34FF34FF348034803479
:102F3C0007340734073407340734073407340734AD
:102F4C000734FF34FF34FF34FF34FF3407340734C5
:102F5C000034E034F834FC34FE34FE341F340F34C7
:102F6C000F340F341F34FF34FE34FE34FC34F03491
:102F7C00003400340034003400348034C034E03485
:102F8C00F034F834FE347F343F341F3407340134CA
:102F9C000034C034F834FC34FF34FF34FF34FF34D5
:102FAC00F934F934F834F834F834F834F834F834B3
:102FBC0020344D3469346B3472346F3463342034C0
:102FCC0037342E3436342E343034203450344934A3
:102FDC00433420343134363446343134363431349D
:0C2FEC003934203420340D340A34003411
:082FF800B03443343B340034D3
:1038C80000348034F034FC34FE34FE343F340F349A
:1038D8000F340F343F34FE34FE34FC34F03480347B
:1038E8000034FF34FF34FF34FF34FF340034003435
:1038F800003400340034FF34FF34FF34FF34FF3425
:10390800003403340F343F347F347F34FC34F034D4
:10391800F034F034FC347F347F343F340F340134D6
:10392800003400340034C034E034E034F034F83487
:103938007C34FE34FF34FF34FF34FF340034003469
:1039480000340034003403340134013400340034CA
:103958000034FF34FF34FF34FF34FF3400340034C4
:1039680000340034003400340034003400340034AF
:103978000034FF34FF34FF34FF34FF3400340034A4
:1039880000341F341F341F341F341F341F341F34B6
:103998001F349F34FF34FF34FF343F341F340F3457
:1039A80000340034003400340034E034F834FC349B
:1039B800FF347F340F3403340034003400340034CF
:1039C800003400340034F034FF34FF34FF34FF3463
:1039D8000734003400340034003400340034003438
:1039E8000034F034FC34FE34FE34FF341F340F341A
:1039F8000F340F341F34FF34FE34FE34FC34F034FB
:103A080000348134C334E734FF34FF347E343C342B
:103A18003C343C347E34FF34FF34E734C3348134DF
:103A280000340F343F347F347F34FF34F834F034BB
:103A3800F034F034F834FF347F347F343F340F34BB
:103A480000348034F034F834FC34FE343E340F341F
:103A58000F340F341F347F347E347E347C3470341A
:103A68000034FF34FF34FF34FF34FF343C341E3459
:103A78001E341E343E34FE34FC34FC34F034E0345E
:103A8800003401340F343F347F347F34F834F03459
:103A9800F034F034F834FF347F343F341F340734C3
:103AA800003400348034FC34FF34FF34FF343F34B6
:103AB8001F341F341F341F341F341F341F34003485
:103AC800003418343F343F343F343F341F340F340C
:103AD8000F340F341F34FF34FE34FE34F834E0342E
:103AE800003406341F343F347F347F34FC34F034E0
:103AF800F034F034F8347F347F343F341F340734E3
:103B0800203444344534563449344334453420341D
:103B18003A3420344F344C3445344434203444341B
:103B28004934533450344C344134593420344934B2
:103B38004934433420344934323443342034303423
:103B48002E3439343134203420343134323438345A
:0E3B580078343334323420340D340A340034DF
:103B66000D340A3420344F34663466347334653485
:103B7600743420346F347534743420346F346634BE
:103B86002034723461346E346734653420342B3417
:103B96002D343334B0344334203428342A34313489
:103BA600303430343034293420340D340A3420345F
:023BB6000034D9
:103BB80020344934323443343134203469346E3457
:103BC8006934743420345234423434343D345334F8
:103BD8004434413420345234423436343D3453343E
:0A3BE80043344C340D340A34003429
:103BF200203449346E3469347434203455344134B9
:103C020052345434313420345234423437343D3413
:103C12005434583420345234423435343D345234DE
:0A3C2200583420340D340A34003405
:103C2C00523465346134643420344F346634663431
:103C3C007334653474342034543465346D347034D6
:103C4C002E3465346E3420344834453446342034B4
:063C5C003A34203400346C
:103C620042346134643420344C3465346334743403
:103C72002E3420344F3466346634733465347434ED
:063C82000D340A34003489
:103C88002034503472346534733465346E3474348B
:103C98006134743469346F346E3420343A340D34FA
:043CA8000A340034A6
:103CAC0020343134723473347434203476346134C7
:103CBC006C347534653420344834453446343D34E2
:043CCC00203400346C
:103CD00030343134323433343434353436343734A8
:103CE000383439344134423443344434453446342E
:103CF00045347234613473346534203423343134C0
:0E3D000020344834453446340D340A3400343F
:103D0E002034463461346D3469346C347934203463
:0E3D1E0043346F34643465343A342034003456
:103D2C005734723469347434653420342334313468
:0E3D3C0020344834453446340D340A34003403
:103D4A004E346534773420344F34663466347334F1
:0C3D5A006534743420343A3420340034D2
:103D66004834453446342034763469346534723404
:0A3D7600673465340D340A3400345C
:103D800020344F344C3445344434203443344C34A0
:0A3D9000533420340D340A3400349B
:103D9A002034423441345634413452344434203489
:083DAA004F344E342034003484
:103DB20020344D346F346434653420344D347534DA
:083DC200653474342034003430
:103DCA002E342E344F344B3420342E342E342034B7
:023DDA000034B3
:103DDC002E342E344234413444340D340A342034DD
:023DEC000034A1
:0E3DEE0020344934443431343D342034003420
:0C3DFC003B342034453463343D34003443
:0C3E080020344F34663473343D340034F1
:083E1400543443343D34003402
:083E1C00543442343D340034FB
:083E240020344F344B3400340C
:063E2C003B342034003499
:020000040001F9
:06000E00E438831E1F3FD1
:00000001FF
